:0600000000008A01122835
:080008000900483465346C3432
:100010006C346F34203477346F3472346C3464341D
:10002000213400348330831681008B1239308312DF
:1000300090006030F8002E201D280530F0000030C0
:10004000F10044200D3038200A303820E830F0002C
:100050000330F10056201D2863002C2867308316DA
:10006000031399001815981683121816981708008C
:10007000831203130C1E3A2899000800700FF10335
:10008000F10AF000710408004B2000380319080041
:1000900038203E20442871088A0070088200F0034E
:1000A000700FF10AF1037008710408000B110B1DA9
:0A00B00057284F20031D56280800B2
:00000001FF
